###############################################################################
#
# IAR ELF Linker V7.50.2.10312/W32 for ARM                06/Aug/2020  18:18:48
# Copyright 2007-2015 IAR Systems AB.
#
#    Output file  =  
#        D:\Projects\MicroTechnics\Projects_site\MT_LIN_SW_Example\EWARM\MT_LIN_SW_Example\Exe\MT_LIN_SW_Example.out
#    Map file     =  
#        D:\Projects\MicroTechnics\Projects_site\MT_LIN_SW_Example\EWARM\MT_LIN_SW_Example\List\MT_LIN_SW_Example.map
#    Command line =  
#        D:\Projects\MicroTechnics\Projects_site\MT_LIN_SW_Example\EWARM\MT_LIN_SW_Example\Obj\lin.o
#        D:\Projects\MicroTechnics\Projects_site\MT_LIN_SW_Example\EWARM\MT_LIN_SW_Example\Obj\main.o
#        D:\Projects\MicroTechnics\Projects_site\MT_LIN_SW_Example\EWARM\MT_LIN_SW_Example\Obj\startup_stm32f103xe.o
#        D:\Projects\MicroTechnics\Projects_site\MT_LIN_SW_Example\EWARM\MT_LIN_SW_Example\Obj\stm32f1xx_hal.o
#        D:\Projects\MicroTechnics\Projects_site\MT_LIN_SW_Example\EWARM\MT_LIN_SW_Example\Obj\stm32f1xx_hal_cortex.o
#        D:\Projects\MicroTechnics\Projects_site\MT_LIN_SW_Example\EWARM\MT_LIN_SW_Example\Obj\stm32f1xx_hal_dma.o
#        D:\Projects\MicroTechnics\Projects_site\MT_LIN_SW_Example\EWARM\MT_LIN_SW_Example\Obj\stm32f1xx_hal_exti.o
#        D:\Projects\MicroTechnics\Projects_site\MT_LIN_SW_Example\EWARM\MT_LIN_SW_Example\Obj\stm32f1xx_hal_flash.o
#        D:\Projects\MicroTechnics\Projects_site\MT_LIN_SW_Example\EWARM\MT_LIN_SW_Example\Obj\stm32f1xx_hal_flash_ex.o
#        D:\Projects\MicroTechnics\Projects_site\MT_LIN_SW_Example\EWARM\MT_LIN_SW_Example\Obj\stm32f1xx_hal_gpio.o
#        D:\Projects\MicroTechnics\Projects_site\MT_LIN_SW_Example\EWARM\MT_LIN_SW_Example\Obj\stm32f1xx_hal_gpio_ex.o
#        D:\Projects\MicroTechnics\Projects_site\MT_LIN_SW_Example\EWARM\MT_LIN_SW_Example\Obj\stm32f1xx_hal_msp.o
#        D:\Projects\MicroTechnics\Projects_site\MT_LIN_SW_Example\EWARM\MT_LIN_SW_Example\Obj\stm32f1xx_hal_pwr.o
#        D:\Projects\MicroTechnics\Projects_site\MT_LIN_SW_Example\EWARM\MT_LIN_SW_Example\Obj\stm32f1xx_hal_rcc.o
#        D:\Projects\MicroTechnics\Projects_site\MT_LIN_SW_Example\EWARM\MT_LIN_SW_Example\Obj\stm32f1xx_hal_rcc_ex.o
#        D:\Projects\MicroTechnics\Projects_site\MT_LIN_SW_Example\EWARM\MT_LIN_SW_Example\Obj\stm32f1xx_hal_tim.o
#        D:\Projects\MicroTechnics\Projects_site\MT_LIN_SW_Example\EWARM\MT_LIN_SW_Example\Obj\stm32f1xx_hal_tim_ex.o
#        D:\Projects\MicroTechnics\Projects_site\MT_LIN_SW_Example\EWARM\MT_LIN_SW_Example\Obj\stm32f1xx_hal_uart.o
#        D:\Projects\MicroTechnics\Projects_site\MT_LIN_SW_Example\EWARM\MT_LIN_SW_Example\Obj\stm32f1xx_it.o
#        D:\Projects\MicroTechnics\Projects_site\MT_LIN_SW_Example\EWARM\MT_LIN_SW_Example\Obj\system_stm32f1xx.o
#        --redirect _Printf=_PrintfFull --redirect _Scanf=_ScanfFull -o
#        D:\Projects\MicroTechnics\Projects_site\MT_LIN_SW_Example\EWARM\MT_LIN_SW_Example\Exe\MT_LIN_SW_Example.out
#        --map
#        D:\Projects\MicroTechnics\Projects_site\MT_LIN_SW_Example\EWARM\MT_LIN_SW_Example\List\MT_LIN_SW_Example.map
#        --config
#        D:\Projects\MicroTechnics\Projects_site\MT_LIN_SW_Example\EWARM/stm32f103xe_flash.icf
#        --semihosting --entry __iar_program_start --vfe
#
###############################################################################

*******************************************************************************
*** RUNTIME MODEL ATTRIBUTES
***

CppFlavor       = *
__SystemLibrary = DLib


*******************************************************************************
*** PLACEMENT SUMMARY
***

"A1":  place at 0x08000000 { ro section .intvec };
"P1":  place in [from 0x08000000 to 0x0807ffff] { ro };
"P2":  place in [from 0x20000000 to 0x2000ffff] { rw, block CSTACK, block HEAP };

  Section            Kind        Address    Size  Object
  -------            ----        -------    ----  ------
"A1":                                      0x130
  .intvec            ro code  0x08000000   0x130  startup_stm32f103xe.o [1]
                            - 0x08000130   0x130

"P1":                                     0x2b1c
  .text              ro code  0x08000130   0x8d0  stm32f1xx_hal_uart.o [1]
  .text              ro code  0x08000a00   0x194  stm32f1xx_hal_msp.o [1]
  .text              ro code  0x08000b94    0xb0  stm32f1xx_hal.o [1]
  .text              ro code  0x08000c44   0x248  stm32f1xx_hal_dma.o [1]
  .text              ro code  0x08000e8c   0x5ec  lin.o [1]
  .text              ro code  0x08001478   0x708  stm32f1xx_hal_rcc.o [1]
  .text              ro code  0x08001b80   0x144  stm32f1xx_hal_cortex.o [1]
  .text              ro code  0x08001cc4     0x6  ABImemclr4.o [4]
  .rodata            const    0x08001cca     0x2  stm32f1xx_hal_rcc.o [1]
  .text              ro code  0x08001ccc   0x478  stm32f1xx_hal_gpio.o [1]
  .text              ro code  0x08002144   0x3ea  stm32f1xx_hal_tim.o [1]
  .text              ro code  0x08002530   0x33e  main.o [1]
  .text              ro code  0x08002870    0x56  ABImemcpy_unaligned.o [4]
  .text              ro code  0x080028c8    0x32  ABImemset48.o [4]
  .text              ro code  0x080028fc    0x56  stm32f1xx_hal_tim_ex.o [1]
  .text              ro code  0x08002954    0x68  system_stm32f1xx.o [1]
  .text              ro code  0x080029bc    0x44  stm32f1xx_it.o [1]
  .text              ro code  0x08002a00    0x40  zero_init3.o [4]
  .text              ro code  0x08002a40    0x2c  copy_init3.o [4]
  .text              ro code  0x08002a6c    0x28  data_init.o [4]
  .iar.init_table    const    0x08002a94    0x24  - Linker created -
  Initializer bytes  const    0x08002ab8    0x20  <for P2-1>
  .text              ro code  0x08002ad8    0x1a  cmain.o [4]
  .text              ro code  0x08002af2     0x4  low_level_init.o [3]
  .text              ro code  0x08002af6     0x4  exit.o [3]
  .text              ro code  0x08002afc     0xa  cexit.o [4]
  .text              ro code  0x08002b08    0x14  exit.o [5]
  .rodata            const    0x08002b1c    0x10  stm32f1xx_hal_rcc.o [1]
  .rodata            const    0x08002b2c    0x10  system_stm32f1xx.o [1]
  .text              ro code  0x08002b3c    0x10  startup_stm32f103xe.o [1]
  .text              ro code  0x08002b4c     0xc  cstartup_M.o [4]
  .rodata            const    0x08002b58     0x8  main.o [1]
  .rodata            const    0x08002b60     0x8  system_stm32f1xx.o [1]
  .text              ro code  0x08002b68     0x4  startup_stm32f103xe.o [1]
  .text              ro code  0x08002b6c     0x4  startup_stm32f103xe.o [1]
  .text              ro code  0x08002b70     0x4  startup_stm32f103xe.o [1]
  .text              ro code  0x08002b74     0x4  startup_stm32f103xe.o [1]
  .text              ro code  0x08002b78     0x4  startup_stm32f103xe.o [1]
  .text              ro code  0x08002b7c     0x4  startup_stm32f103xe.o [1]
  .text              ro code  0x08002b80     0x4  startup_stm32f103xe.o [1]
  .text              ro code  0x08002b84     0x4  startup_stm32f103xe.o [1]
  .text              ro code  0x08002b88     0x4  startup_stm32f103xe.o [1]
  .text              ro code  0x08002b8c     0x4  startup_stm32f103xe.o [1]
  .text              ro code  0x08002b90     0x4  startup_stm32f103xe.o [1]
  .text              ro code  0x08002b94     0x4  startup_stm32f103xe.o [1]
  .text              ro code  0x08002b98     0x4  startup_stm32f103xe.o [1]
  .text              ro code  0x08002b9c     0x4  startup_stm32f103xe.o [1]
  .text              ro code  0x08002ba0     0x4  startup_stm32f103xe.o [1]
  .text              ro code  0x08002ba4     0x4  startup_stm32f103xe.o [1]
  .text              ro code  0x08002ba8     0x4  startup_stm32f103xe.o [1]
  .text              ro code  0x08002bac     0x4  startup_stm32f103xe.o [1]
  .text              ro code  0x08002bb0     0x4  startup_stm32f103xe.o [1]
  .text              ro code  0x08002bb4     0x4  startup_stm32f103xe.o [1]
  .text              ro code  0x08002bb8     0x4  startup_stm32f103xe.o [1]
  .text              ro code  0x08002bbc     0x4  startup_stm32f103xe.o [1]
  .text              ro code  0x08002bc0     0x4  startup_stm32f103xe.o [1]
  .text              ro code  0x08002bc4     0x4  startup_stm32f103xe.o [1]
  .text              ro code  0x08002bc8     0x4  startup_stm32f103xe.o [1]
  .text              ro code  0x08002bcc     0x4  startup_stm32f103xe.o [1]
  .text              ro code  0x08002bd0     0x4  startup_stm32f103xe.o [1]
  .text              ro code  0x08002bd4     0x4  startup_stm32f103xe.o [1]
  .text              ro code  0x08002bd8     0x4  startup_stm32f103xe.o [1]
  .text              ro code  0x08002bdc     0x4  startup_stm32f103xe.o [1]
  .text              ro code  0x08002be0     0x4  startup_stm32f103xe.o [1]
  .text              ro code  0x08002be4     0x4  startup_stm32f103xe.o [1]
  .text              ro code  0x08002be8     0x4  startup_stm32f103xe.o [1]
  .text              ro code  0x08002bec     0x4  startup_stm32f103xe.o [1]
  .text              ro code  0x08002bf0     0x4  startup_stm32f103xe.o [1]
  .text              ro code  0x08002bf4     0x4  startup_stm32f103xe.o [1]
  .text              ro code  0x08002bf8     0x4  startup_stm32f103xe.o [1]
  .text              ro code  0x08002bfc     0x4  startup_stm32f103xe.o [1]
  .text              ro code  0x08002c00     0x4  startup_stm32f103xe.o [1]
  .text              ro code  0x08002c04     0x4  startup_stm32f103xe.o [1]
  .text              ro code  0x08002c08     0x4  startup_stm32f103xe.o [1]
  .text              ro code  0x08002c0c     0x4  startup_stm32f103xe.o [1]
  .text              ro code  0x08002c10     0x4  startup_stm32f103xe.o [1]
  .text              ro code  0x08002c14     0x4  startup_stm32f103xe.o [1]
  .text              ro code  0x08002c18     0x4  startup_stm32f103xe.o [1]
  .text              ro code  0x08002c1c     0x4  startup_stm32f103xe.o [1]
  .text              ro code  0x08002c20     0x4  startup_stm32f103xe.o [1]
  .text              ro code  0x08002c24     0x4  startup_stm32f103xe.o [1]
  .text              ro code  0x08002c28     0x4  startup_stm32f103xe.o [1]
  .text              ro code  0x08002c2c     0x4  startup_stm32f103xe.o [1]
  .text              ro code  0x08002c30     0x4  startup_stm32f103xe.o [1]
  .text              ro code  0x08002c34     0x4  startup_stm32f103xe.o [1]
  .text              ro code  0x08002c38     0x4  startup_stm32f103xe.o [1]
  .text              ro code  0x08002c3c     0x4  startup_stm32f103xe.o [1]
  .text              ro code  0x08002c40     0x4  startup_stm32f103xe.o [1]
  .text              ro code  0x08002c44     0x4  startup_stm32f103xe.o [1]
  .text              ro code  0x08002c48     0x4  startup_stm32f103xe.o [1]
  .rodata            const    0x08002c4c     0x0  zero_init3.o [4]
  .rodata            const    0x08002c4c     0x0  copy_init3.o [4]
                            - 0x08002c4c  0x2b1c

"P2", part 1 of 3:                          0x20
  P2-1                        0x20000000    0x1f  <Init block>
    .data            inited   0x20000000     0x8  main.o [1]
    .data            inited   0x20000008     0x8  main.o [1]
    .data            inited   0x20000010     0x4  stm32f1xx_hal.o [1]
    .data            inited   0x20000014     0x4  system_stm32f1xx.o [1]
    .data            inited   0x20000018     0x2  lin.o [1]
    .data            inited   0x2000001a     0x1  lin.o [1]
    .data            inited   0x2000001b     0x1  main.o [1]
    .data            inited   0x2000001c     0x1  main.o [1]
    .data            inited   0x2000001d     0x1  main.o [1]
    .data            inited   0x2000001e     0x1  stm32f1xx_hal.o [1]
                            - 0x2000001f    0x1f

"P2", part 2 of 3:                         0x400
  CSTACK                      0x20000020   0x400  <Block>
    CSTACK           uninit   0x20000020   0x400  <Block tail>
                            - 0x20000420   0x400

"P2", part 3 of 3:                         0x118
  .bss               zero     0x20000420    0x40  main.o [1]
  .bss               zero     0x20000460    0x40  main.o [1]
  .bss               zero     0x200004a0    0x40  main.o [1]
  .bss               zero     0x200004e0     0x8  main.o [1]
  .bss               zero     0x200004e8     0x8  main.o [1]
  .bss               zero     0x200004f0     0x4  lin.o [1]
  .bss               zero     0x200004f4     0x4  lin.o [1]
  .bss               zero     0x200004f8     0x4  lin.o [1]
  .bss               zero     0x200004fc     0x4  lin.o [1]
  .bss               zero     0x20000500     0x4  lin.o [1]
  .bss               zero     0x20000504     0x4  lin.o [1]
  .bss               zero     0x20000508     0x4  lin.o [1]
  .bss               zero     0x2000050c     0x4  lin.o [1]
  .bss               zero     0x20000510     0x4  main.o [1]
  .bss               zero     0x20000514     0x4  main.o [1]
  .bss               zero     0x20000518     0x4  main.o [1]
  .bss               zero     0x2000051c     0x4  main.o [1]
  .bss               zero     0x20000520     0x4  stm32f1xx_hal.o [1]
  .bss               zero     0x20000524     0x2  lin.o [1]
  .bss               zero     0x20000526     0x2  lin.o [1]
  .bss               zero     0x20000528     0x2  lin.o [1]
  .bss               zero     0x2000052a     0x2  lin.o [1]
  .bss               zero     0x2000052c     0x2  lin.o [1]
  .bss               zero     0x2000052e     0x1  lin.o [1]
  .bss               zero     0x2000052f     0x1  lin.o [1]
  .bss               zero     0x20000530     0x1  lin.o [1]
  .bss               zero     0x20000531     0x1  lin.o [1]
  .bss               zero     0x20000532     0x1  lin.o [1]
  .bss               zero     0x20000533     0x1  lin.o [1]
  .bss               zero     0x20000534     0x1  lin.o [1]
  .bss               zero     0x20000535     0x1  lin.o [1]
  .bss               zero     0x20000536     0x1  main.o [1]
                            - 0x20000537   0x117


*******************************************************************************
*** INIT TABLE
***

          Address     Size
          -------     ----
Zero (__iar_zero_init3)
    1 destination range, total size 0x117:
          0x20000420  0x117

Copy (__iar_copy_init3)
    1 source range, total size 0x20 (103% of destination):
          0x08002ab8   0x20
    1 destination range, total size 0x1f:
          0x20000000   0x1f



*******************************************************************************
*** MODULE SUMMARY
***

    Module                  ro code  ro data  rw data
    ------                  -------  -------  -------
D:\Projects\MicroTechnics\Projects_site\MT_LIN_SW_Example\EWARM\MT_LIN_SW_Example\Obj: [1]
    lin.o                     1 516        3       53
    main.o                      830       27      244
    startup_stm32f103xe.o       548
    stm32f1xx_hal.o             176        5        9
    stm32f1xx_hal_cortex.o      324
    stm32f1xx_hal_dma.o         584
    stm32f1xx_hal_gpio.o      1 144
    stm32f1xx_hal_msp.o         404
    stm32f1xx_hal_rcc.o       1 800       18
    stm32f1xx_hal_tim.o       1 002
    stm32f1xx_hal_tim_ex.o       86
    stm32f1xx_hal_uart.o      2 256
    stm32f1xx_it.o               68
    system_stm32f1xx.o          104       28        4
    -------------------------------------------------
    Total:                   10 842       81      310

command line: [2]
    -------------------------------------------------
    Total:

dl7M_tln.a: [3]
    exit.o                        4
    low_level_init.o              4
    -------------------------------------------------
    Total:                        8

rt7M_tl.a: [4]
    ABImemclr4.o                  6
    ABImemcpy_unaligned.o        86
    ABImemset48.o                50
    cexit.o                      10
    cmain.o                      26
    copy_init3.o                 44
    cstartup_M.o                 12
    data_init.o                  40
    zero_init3.o                 64
    -------------------------------------------------
    Total:                      338

shb_l.a: [5]
    exit.o                       20
    -------------------------------------------------
    Total:                       20

    Gaps                         14
    Linker created                        37    1 024
-----------------------------------------------------
    Grand Total:             11 222      118    1 334


*******************************************************************************
*** ENTRY LIST
***

Entry                      Address   Size  Type      Object
-----                      -------   ----  ----      ------
.iar.init_table$$Base   0x08002a94          --   Gb  - Linker created -
.iar.init_table$$Limit  0x08002ab8          --   Gb  - Linker created -
?main                   0x08002ad9         Code  Gb  cmain.o [4]
AHBPrescTable           0x08002b2c   0x10  Data  Gb  system_stm32f1xx.o [1]
APBPrescTable           0x08002b60    0x8  Data  Gb  system_stm32f1xx.o [1]
BusFault_Handler        0x080029c3    0x2  Code  Gb  stm32f1xx_it.o [1]
CSTACK$$Base            0x20000020          --   Gb  - Linker created -
CSTACK$$Limit           0x20000420          --   Gb  - Linker created -
DebugMon_Handler        0x080029c9    0x2  Code  Gb  stm32f1xx_it.o [1]
Error_Handler           0x0800286d    0x2  Code  Gb  main.o [1]
HAL_DMA_Abort           0x08000c45   0x4e  Code  Gb  stm32f1xx_hal_dma.o [1]
HAL_DMA_Abort_IT        0x08000c93  0x1be  Code  Gb  stm32f1xx_hal_dma.o [1]
HAL_DMA_GetError        0x08000e89    0x4  Code  Gb  stm32f1xx_hal_dma.o [1]
HAL_Delay               0x08000c0d   0x24  Code  Wk  stm32f1xx_hal.o [1]
HAL_GPIO_DeInit         0x08001f9f  0x132  Code  Gb  stm32f1xx_hal_gpio.o [1]
HAL_GPIO_Init           0x08001ccd  0x2d2  Code  Gb  stm32f1xx_hal_gpio.o [1]
HAL_GPIO_ReadPin        0x080020d1   0x18  Code  Gb  stm32f1xx_hal_gpio.o [1]
HAL_GPIO_WritePin       0x080020e9   0x14  Code  Gb  stm32f1xx_hal_gpio.o [1]
HAL_GetTick             0x08000c07    0x6  Code  Wk  stm32f1xx_hal.o [1]
HAL_IncTick             0x08000bf7   0x10  Code  Wk  stm32f1xx_hal.o [1]
HAL_Init                0x08000b95   0x22  Code  Gb  stm32f1xx_hal.o [1]
HAL_InitTick            0x08000bb7   0x40  Code  Wk  stm32f1xx_hal.o [1]
HAL_LIN_Init            0x080001a7   0x94  Code  Gb  stm32f1xx_hal_uart.o [1]
HAL_LIN_SendBreak       0x08000675   0x36  Code  Gb  stm32f1xx_hal_uart.o [1]
HAL_MspInit             0x08000a01   0x48  Code  Gb  stm32f1xx_hal_msp.o [1]
HAL_NVIC_EnableIRQ      0x08001c89    0xe  Code  Gb  stm32f1xx_hal_cortex.o [1]
HAL_NVIC_SetPriority    0x08001c63   0x26  Code  Gb  stm32f1xx_hal_cortex.o [1]
HAL_NVIC_SetPriorityGrouping
                        0x08001c57    0xc  Code  Gb  stm32f1xx_hal_cortex.o [1]
HAL_RCC_ClockConfig     0x080018f9  0x16e  Code  Gb  stm32f1xx_hal_rcc.o [1]
HAL_RCC_GetHCLKFreq     0x08001adf    0x6  Code  Gb  stm32f1xx_hal_rcc.o [1]
HAL_RCC_GetPCLK1Freq    0x08001ae5   0x16  Code  Gb  stm32f1xx_hal_rcc.o [1]
HAL_RCC_GetPCLK2Freq    0x08001afb   0x16  Code  Gb  stm32f1xx_hal_rcc.o [1]
HAL_RCC_GetSysClockFreq
                        0x08001a67   0x78  Code  Gb  stm32f1xx_hal_rcc.o [1]
HAL_RCC_OscConfig       0x08001479  0x480  Code  Gb  stm32f1xx_hal_rcc.o [1]
HAL_SYSTICK_Config      0x08001c97    0xc  Code  Gb  stm32f1xx_hal_cortex.o [1]
HAL_TIMEx_BreakCallback
                        0x08002951    0x2  Code  Wk  stm32f1xx_hal_tim_ex.o [1]
HAL_TIMEx_CommutCallback
                        0x0800294f    0x2  Code  Wk  stm32f1xx_hal_tim_ex.o [1]
HAL_TIMEx_MasterConfigSynchronization
                        0x080028fd   0x52  Code  Gb  stm32f1xx_hal_tim_ex.o [1]
HAL_TIM_Base_Init       0x08002145   0x38  Code  Gb  stm32f1xx_hal_tim.o [1]
HAL_TIM_Base_MspInit    0x08000a49   0x38  Code  Gb  stm32f1xx_hal_msp.o [1]
HAL_TIM_Base_Start_IT   0x0800217d   0x2c  Code  Gb  stm32f1xx_hal_tim.o [1]
HAL_TIM_ConfigClockSource
                        0x0800231f   0xee  Code  Gb  stm32f1xx_hal_tim.o [1]
HAL_TIM_IC_CaptureCallback
                        0x0800240f    0x2  Code  Wk  stm32f1xx_hal_tim.o [1]
HAL_TIM_IRQHandler      0x080021a9  0x176  Code  Gb  stm32f1xx_hal_tim.o [1]
HAL_TIM_OC_DelayElapsedCallback
                        0x0800240d    0x2  Code  Wk  stm32f1xx_hal_tim.o [1]
HAL_TIM_PWM_PulseFinishedCallback
                        0x08002411    0x2  Code  Wk  stm32f1xx_hal_tim.o [1]
HAL_TIM_PeriodElapsedCallback
                        0x080013d7   0x16  Code  Gb  lin.o [1]
HAL_TIM_TriggerCallback
                        0x08002413    0x2  Code  Wk  stm32f1xx_hal_tim.o [1]
HAL_UART_AbortReceive   0x080004c7   0x66  Code  Gb  stm32f1xx_hal_uart.o [1]
HAL_UART_ErrorCallback  0x08000673    0x2  Code  Wk  stm32f1xx_hal_uart.o [1]
HAL_UART_IRQHandler     0x0800052d  0x146  Code  Gb  stm32f1xx_hal_uart.o [1]
HAL_UART_Init           0x08000131   0x76  Code  Gb  stm32f1xx_hal_uart.o [1]
HAL_UART_MspInit        0x08000a81   0xf8  Code  Gb  stm32f1xx_hal_msp.o [1]
HAL_UART_Receive        0x08000319   0xe6  Code  Gb  stm32f1xx_hal_uart.o [1]
HAL_UART_Receive_IT     0x08000457   0x70  Code  Gb  stm32f1xx_hal_uart.o [1]
HAL_UART_RxCpltCallback
                        0x08001403   0x16  Code  Gb  lin.o [1]
HAL_UART_Transmit       0x0800023b   0xde  Code  Gb  stm32f1xx_hal_uart.o [1]
HAL_UART_Transmit_IT    0x080003ff   0x58  Code  Gb  stm32f1xx_hal_uart.o [1]
HAL_UART_TxCpltCallback
                        0x080013ed   0x16  Code  Gb  lin.o [1]
HardFault_Handler       0x080029bf    0x2  Code  Gb  stm32f1xx_it.o [1]
LIN_CalcCheckSum        0x0800114b   0x2e  Code  Gb  lin.o [1]
LIN_GetDataLength       0x08001179   0x2a  Code  Gb  lin.o [1]
LIN_Init                0x08000f3f   0xca  Code  Gb  lin.o [1]
LIN_ReadRxPortState     0x08000e8d   0x18  Code  Gb  lin.o [1]
LIN_Receive             0x080010a5   0x9c  Code  Gb  lin.o [1]
LIN_Reset               0x08001141    0xa  Code  Gb  lin.o [1]
LIN_RxCpltCallback      0x0800280b    0xc  Code  Gb  main.o [1]
LIN_SlaveIdRxCallback   0x080027c5   0x46  Code  Gb  main.o [1]
LIN_TimerProcess        0x080011a3  0x100  Code  Gb  lin.o [1]
LIN_Transmit            0x08001009   0x9c  Code  Gb  lin.o [1]
LIN_UartProcess         0x080012a3  0x134  Code  Gb  lin.o [1]
LIN_WriteTxPortState    0x08000ea5   0x9a  Code  Gb  lin.o [1]
MX_GPIO_Init            0x080027a7   0x1e  Code  Lc  main.o [1]
MX_TIM4_Init            0x080026a9   0x7a  Code  Lc  main.o [1]
MX_USART1_UART_Init     0x08002723   0x40  Code  Lc  main.o [1]
MX_USART2_UART_Init     0x08002763   0x44  Code  Lc  main.o [1]
MemManage_Handler       0x080029c1    0x2  Code  Gb  stm32f1xx_it.o [1]
NMI_Handler             0x080029bd    0x2  Code  Gb  stm32f1xx_it.o [1]
NVIC_EncodePriority     0x08001be9   0x3e  Code  Lc  stm32f1xx_hal_cortex.o [1]
PendSV_Handler          0x080029cb    0x2  Code  Gb  stm32f1xx_it.o [1]
RCC_Delay               0x08001b11   0x26  Code  Lc  stm32f1xx_hal_rcc.o [1]
Region$$Table$$Base     0x08002a94          --   Gb  - Linker created -
Region$$Table$$Limit    0x08002ab8          --   Gb  - Linker created -
SVC_Handler             0x080029c7    0x2  Code  Gb  stm32f1xx_it.o [1]
SysTick_Config          0x08001c27   0x30  Code  Lc  stm32f1xx_hal_cortex.o [1]
SysTick_Handler         0x080029cd    0x8  Code  Gb  stm32f1xx_it.o [1]
SystemClock_Config      0x0800263b   0x6e  Code  Gb  main.o [1]
SystemCoreClock         0x20000014    0x4  Data  Gb  system_stm32f1xx.o [1]
SystemInit              0x08002955   0x4e  Code  Gb  system_stm32f1xx.o [1]
TIM4_IRQHandler         0x080029d5    0xa  Code  Gb  stm32f1xx_it.o [1]
TIM_Base_SetConfig      0x08002415   0x88  Code  Gb  stm32f1xx_hal_tim.o [1]
TIM_ETR_SetConfig       0x08002515   0x1a  Code  Gb  stm32f1xx_hal_tim.o [1]
TIM_ITRx_SetConfig      0x08002503   0x12  Code  Lc  stm32f1xx_hal_tim.o [1]
TIM_TI1_ConfigInputStage
                        0x080024b1   0x28  Code  Lc  stm32f1xx_hal_tim.o [1]
TIM_TI2_ConfigInputStage
                        0x080024d9   0x2a  Code  Lc  stm32f1xx_hal_tim.o [1]
UART_DMAAbortOnError    0x0800073d   0x16  Code  Lc  stm32f1xx_hal_uart.o [1]
UART_EndRxTransfer      0x0800071b   0x20  Code  Lc  stm32f1xx_hal_uart.o [1]
UART_EndTransmit_IT     0x080007c3   0x20  Code  Lc  stm32f1xx_hal_uart.o [1]
UART_Receive_IT         0x080007e3   0xac  Code  Lc  stm32f1xx_hal_uart.o [1]
UART_SetConfig          0x0800088f  0x16a  Code  Lc  stm32f1xx_hal_uart.o [1]
UART_Transmit_IT        0x08000755   0x6e  Code  Lc  stm32f1xx_hal_uart.o [1]
UART_WaitOnFlagUntilTimeout
                        0x080006ab   0x70  Code  Lc  stm32f1xx_hal_uart.o [1]
USART1_IRQHandler       0x080029df    0xa  Code  Gb  stm32f1xx_it.o [1]
USART2_IRQHandler       0x080029e9    0xa  Code  Gb  stm32f1xx_it.o [1]
UsageFault_Handler      0x080029c5    0x2  Code  Gb  stm32f1xx_it.o [1]
__NVIC_EnableIRQ        0x08001ba9   0x1a  Code  Lc  stm32f1xx_hal_cortex.o [1]
__NVIC_GetPriorityGrouping
                        0x08001b9f    0xa  Code  Lc  stm32f1xx_hal_cortex.o [1]
__NVIC_SetPriority      0x08001bc3   0x26  Code  Lc  stm32f1xx_hal_cortex.o [1]
__NVIC_SetPriorityGrouping
                        0x08001b81   0x1e  Code  Lc  stm32f1xx_hal_cortex.o [1]
__aeabi_memclr4         0x08001cc5         Code  Gb  ABImemclr4.o [4]
__cmain                 0x08002ad9         Code  Gb  cmain.o [4]
__exit                  0x08002b09   0x14  Code  Gb  exit.o [5]
__iar_Memset4_word      0x080028c9         Code  Gb  ABImemset48.o [4]
__iar_Memset8_word      0x080028c9         Code  Gb  ABImemset48.o [4]
__iar_copy_init3        0x08002a41   0x2c  Code  Gb  copy_init3.o [4]
__iar_data_init3        0x08002a6d   0x28  Code  Gb  data_init.o [4]
__iar_program_start     0x08002b4d         Code  Gb  cstartup_M.o [4]
__iar_unaligned___aeabi_memcpy4
                        0x08002871         Code  Gb  ABImemcpy_unaligned.o [4]
__iar_unaligned___aeabi_memcpy8
                        0x08002871         Code  Gb  ABImemcpy_unaligned.o [4]
__iar_zero_init3        0x08002a01   0x40  Code  Gb  zero_init3.o [4]
__low_level_init        0x08002af3    0x4  Code  Gb  low_level_init.o [3]
__vector_table          0x08000000         Data  Gb  startup_stm32f103xe.o [1]
_call_main              0x08002ae5         Code  Gb  cmain.o [4]
_exit                   0x08002afd         Code  Gb  cexit.o [4]
_main                   0x08002aef         Code  Gb  cmain.o [4]
breakCnt                0x20000524    0x2  Data  Lc  lin.o [1]
breakCntLimit           0x20000526    0x2  Data  Lc  lin.o [1]
breakCntLowerLimit      0x2000052a    0x2  Data  Lc  lin.o [1]
breakCntUpperLimit      0x20000528    0x2  Data  Lc  lin.o [1]
curBaudrate             0x200004f0    0x4  Data  Lc  lin.o [1]
curMode                 0x2000052f    0x1  Data  Lc  lin.o [1]
curState                0x2000052e    0x1  Data  Lc  lin.o [1]
dataPtr                 0x200004f4    0x4  Data  Lc  lin.o [1]
exit                    0x08002af7    0x4  Code  Gb  exit.o [3]
htim4                   0x20000420   0x40  Data  Gb  main.o [1]
huart1                  0x20000460   0x40  Data  Gb  main.o [1]
huart2                  0x200004a0   0x40  Data  Gb  main.o [1]
isInit                  0x20000535    0x1  Data  Lc  lin.o [1]
linMasterRequestCnt     0x20000518    0x4  Data  Gb  main.o [1]
linMasterRxCnt          0x2000051c    0x4  Data  Gb  main.o [1]
linMasterRxData         0x200004e0    0x8  Data  Gb  main.o [1]
linMasterTask           0x20000536    0x1  Data  Gb  main.o [1]
linMasterTxCnt          0x20000510    0x4  Data  Gb  main.o [1]
linMasterTxData         0x20000000    0x8  Data  Gb  main.o [1]
linRxId                 0x2000001d    0x1  Data  Gb  main.o [1]
linSlaveRxCnt           0x20000514    0x4  Data  Gb  main.o [1]
linSlaveRxData          0x200004e8    0x8  Data  Gb  main.o [1]
linSlaveTxData          0x20000008    0x8  Data  Gb  main.o [1]
linSync                 0x2000001b    0x1  Data  Gb  main.o [1]
linTxId                 0x2000001c    0x1  Data  Gb  main.o [1]
main                    0x08002531  0x10a  Code  Gb  main.o [1]
rxByte                  0x20000534    0x1  Data  Lc  lin.o [1]
rxDataNum               0x20000531    0x1  Data  Lc  lin.o [1]
rxPin                   0x20000508    0x4  Data  Lc  lin.o [1]
rxPort                  0x20000500    0x4  Data  Lc  lin.o [1]
rxTimeoutCnt            0x2000052c    0x2  Data  Lc  lin.o [1]
rxTimeoutCntLimit       0x20000018    0x2  Data  Lc  lin.o [1]
syncByte                0x2000001a    0x1  Data  Lc  lin.o [1]
timerHandle             0x200004fc    0x4  Data  Lc  lin.o [1]
txCheckSum              0x20000533    0x1  Data  Lc  lin.o [1]
txDataNum               0x20000530    0x1  Data  Lc  lin.o [1]
txId                    0x20000532    0x1  Data  Lc  lin.o [1]
txPin                   0x2000050c    0x4  Data  Lc  lin.o [1]
txPort                  0x20000504    0x4  Data  Lc  lin.o [1]
uartHandle              0x200004f8    0x4  Data  Lc  lin.o [1]
uwTick                  0x20000520    0x4  Data  Gb  stm32f1xx_hal.o [1]
uwTickFreq              0x2000001e    0x1  Data  Gb  stm32f1xx_hal.o [1]
uwTickPrio              0x20000010    0x4  Data  Gb  stm32f1xx_hal.o [1]


[1] = D:\Projects\MicroTechnics\Projects_site\MT_LIN_SW_Example\EWARM\MT_LIN_SW_Example\Obj
[2] = command line
[3] = dl7M_tln.a
[4] = rt7M_tl.a
[5] = shb_l.a

  11 222 bytes of readonly  code memory
     118 bytes of readonly  data memory
   1 334 bytes of readwrite data memory

Errors: none
Warnings: none
